:101E3900AF5FEFC4135407FFEF30E032E5277016A8
:101E4900E5287012E529700EAF5EEF54EFF55EAF2D
:101E59005EEF54F7F55EE52E6005E52EB480087F48
:0F1E6900017E00120BCF227F007E00120BCF22D2
:040BCF008E418F4282
:100BD300E54245417003020CCDAF34EFC413135407
:100BE30003FFEF20E020AF33EF131313541FFFEF86
:100BF30020E013AF5DEFC413135403FFEF20E006AF
:100C0300AF34EF30E0D3C2AFAF34EF54BFF534D2DB
:100C1300AF90702C7404F09070587402F0AE37AF3C
:100C230038E4FCFDAB3EAA3DA93CA83BD3121563B7
:100C330040088537438538448008AE3DAF3E8E4338
:100C43008F44AF5FEF30E028756000756100C3E546
:100C5300619544E5609543503D907020E0FFAE619F
:100C630074662EF8A6070561E5617002056080DEF3
:100C7300756000756100C3E5619544E56095435077
:100C830015907020E0FF7E008E5A8F5B0561E56151
:100C93007002056080E0AE43AF44AB07AA06E4F9F7
:100CA300F8C3E53E9BF53EE53D9AF53DE53C99F5F8
:100CB3003CE53B98F53BAF3EAE3DAD3CAC3BEC4D2C
:100CC3004E4F6003020BDC020DF390702C7405F0A1
:100CD3009070587402F0AE37AF38E4FCFDAB3EAA17
:100CE3003DA93CA83BD31215634019AF3890701C43
:100CF300EFF0E537FF7E0090701DEFF085374385F9
:100D030038448021AF3E90701CEFF0AF3EAE3DAD56
:100D13003CAC3B780812157490701DEFF0AE3DAFFC
:100D23003E8E438F44AF5FEF30E0287560007561FE
:100D330000C3E5619544E5609543503BAF6174663C
:100D43002FF8E6FF907020EFF00561E56170020572
:100D53006080DE756000756100C3E5619544E56000
:100D6300954350137E00AF61907020EFF00561E56D
:100D7300617002056080E2AF34EFC41313135401B2
:100D8300FFEF20E020AF33EF131313541FFFEF20C7
:100D9300E013AF5DEFC413135403FFEF20E006AF7E
:100DA30034EF30E0D2C2AFAF34EF547FF534D2AF7B
:100DB300AE43AF44AB07AA06E4F9F8C3E53E9BF59F
:100DC3003EE53D9AF53DE53C99F53CE53B98F53B21
:100DD300AF3EAE3DAD3CAC3BEC4D4E4F6003020C21
:100DE300CDC294AF1AEF54FEF51A75600075610019
:070DF300AF5FEF54DFF55F75
:010DFA0022D6
:0421630002157000F1
:1016BA00758E02758F01753E00753D00753C00758B
:1016CA003B00753700753840751400AF25EF54009C
:1016DA00FFEF4404F525121F0F90700CE0FFEF5442
:1016EA00FEFF90700CEFF0C2B47F647E00121BC83C
:1016FA00D2B47F647E00121BC8AE15AF168F828EDD
:10170A0083E5822471F582E5833400F583E0FFEFF7
:10171A00B481D4AE15AF168F828E83E5822472F51A
:10172A0082E5833400F583E0FFEFB415BA7536001D
:10173A00753500753400753300751900751A007512
:10174A005F00755E00755D00755C00AF5FEF440178
:08175A00F55FC290121FC222CC
:101F0F007589117510077511D075124E75132075DF
:101F1F008B50758D3C758800C2AF75A803D2AB7519
:0E1F2F00B800D2BBD2B9D2AFD28E7587402295
:101FC200122073120916AF23EF541FF523751B005D
:101FD200AF26EF54FEF526AF26EF4440F526AF5E5E
:081FE200EF54DFF55ED2A822E6
:1020730090700CE0FFEF448CFF90700CEFF09070C9
:0F208300107454F09070141215A639FD0000224D
:10091600AF5FEF20E003020A6F90702C7402F09034
:1009260070047440F0A3E4F090702C7403F090709F
:10093600047440F0A3E4F090702C7404F0907004FA
:100946007440F0A3E4F090702C7405F09070047479
:1009560040F0A3E4F090702C7406F090700474409C
:10096600F0A3E4F090702C7407F09070047440F0DB
:10097600A3E4F090702C7402F09070087417F0A342
:10098600E4F090702C7403F09070087417F0A3E4F0
:10099600F090702C7404F09070087416F0A3E4F0D4
:1009A60090702C7405F09070087416F0A3E4F09023
:1009B600702C7406F09070087415F0A3E4F0907033
:1009C6002C7407F09070087415F0A3E4F090702C66
:1009D6007402F0907008E0FEA3E0FFEE4408FE907B
:1009E6007008EEF0A3EFF090702C7403F09070088E
:1009F600E0FEA3E0FFEE4408FE907008EEF0A3EFE1
:100A0600F090702C7404F0907008E0FEA3E0FFEE06
:100A16004408FE907008EEF0A3EFF090702C740579
:100A2600F0907008E0FEA3E0FFEE4408FE90700828
:100A3600EEF0A3EFF090702C7406F0907008E0FED4
:100A4600A3E0FFEE4408FE907008EEF0A3EFF090EE
:100A5600702C7407F0907008E0FEA3E0FFEE4408E7
:100A6600FE907008EEF0A3EFF0AF5FEF30E0030208
:100A76000BC890702C7402F09070047440F0A3E4DC
:100A8600F090702C7403F09070047440F0A3E4F0BE
:100A960090702C7404F0907004E4F0A37402F0904B
:100AA600702C7405F0907004E4F0A37402F090705A
:100AB6002C7406F09070047440F0A3E4F090702C4F
:100AC6007407F09070047440F0A3E4F090702C74F6
:100AD60002F09070087417F0A3E4F090702C740381
:100AE600F09070087417F0A3E4F090702C7404F082
:100AF6009070087416F0A3E4F090702C7405F090D2
:100B060070087416F0A3E4F090702C7406F09070E0
:100B1600087415F0A3E4F090702C7407F090700838
:100B26007415F0A3E4F090702C7402F0907008E055
:100B3600FEA3E0FFEE4408FE907008EEF0A3EFF08F
:100B460090702C7403F0907008E0FEA3E0FFEE4472
:100B560008FE907008EEF0A3EFF090702C7404F08D
:100B6600907008E0FEA3E0FFEE4408FE907008EEE9
:100B7600F0A3EFF090702C7405F0907008E0FEA3DF
:100B8600E0FFEE4408FE907008EEF0A3EFF09070E0
:100B96002C7406F0907008E0FEA3E0FFEE4408FE19
:100BA600907008EEF0A3EFF090702C7407F0907040
:100BB60008E0FEA3E0FFEE4408FE907008EEF0A306
:090BC600EFF09070007480F02241
:032167000159001B
:03001300020006E2
:0100060032C7
:03001B0002215A65
:09215A00758D3C758B500559325E
:03002300020007D1
:0100070032C6
:03002B00020008C8
:0100080032C5
:03000B00022129A6
:10212900C0E0C0D075D000AF5DEF4420F55DD0D0E0
:03213900D0E032C1
:03000300021A617D
:101A6100C0E0C0F0C083C082C0D075D008907018AB
:101A7100E0FCA3E0FDA3E0FEA3E0FFE5364FF53671
:101A8100E5354EF535E5344DF534E5334CF533AFF9
:101A910036AE35AD34AC3390701812159AAF33EFC2
:101AA10030E02EAF33EF54FEF533AF5DEF4440F538
:101AB1005D753700753840C290AF5FEF4401F55F47
:101AC100121FC290700CE0FFEF4401FF90700CEF09
:0C1AD100F0D0D0D082D083D0F0D0E03232
:0D214D0000124830120000000000000000E9
:10160A007F05121F6B7BFF7A2179527D08121E78A3
:10161A001216BA90700CE0FFEF4401FF90700CEFC5
:10162A00F0121762121E39AF34EFC4540FFFEF30B5
:10163A00E0267B007A0079667D087C007F02121A18
:10164A00DD7F01121F6B7B007A0079667D08121E0E
:10165A0078AF34EF54EFF534E559B41EC47F011264
:10166A001F6B1220B17866A6077866E6FFEF700650
:10167A00786676FF80037866167F01121F6B7B00FF
:10168A007A0079677547037D027FA2121B53786936
:10169A00E6FFEF543FFF7869A6077B007A00796678
:1016AA007D047C007F03121CEC75591402162B2250
:021F6B008F41A4
:101F6D00E541D394004020754200E542C39464508E
:101F7D0012754300E543C394645004054380F50591
:091F8D004280E7154180D97F0074
:011F96002228
:101BC8008E418F4285105A85115BC374FF955BF572
:101BD8005B74FF955AF55AD2A9E55AF55B755A0018
:101BE800855B8C85105A85115BC374FF955BF55B2B
:101BF80074FF955AF55A855B8AD28CAF5DEF54DF36
:101C0800F55DAF5DEFC4135407FFEF30E0F4AF5D4F
:101C1800EF54DFF55DC28CC2A9E54215427002158A
:081C280041E5424541709D2297
:1012A8001201100100000040CC04491B000001029B
:1012B80000011201000200000040CC04491B00009C
:1012C800010200010A0600020000004001000902B4
:1012D8002E00010100C03209072E00010100C032B2
:1012E80009040000040000000009040000040000D4
:1012F80000000705020240000007058202400000C6
:101308000705020200020007058202000200070525
:10131800010340000107058103400001070501039F
:101328004000010705810340000109040001020093
:101338000000000705030140000107058301400084
:1013480001070503010000010705830100000130C2
:10135800035000680069006C006900700073002089
:10136800004900530050003100350038003100209A
:1013780000560065007200200031002E0030000089
:101388000000000000000000000000000000001C39
:10139800035000680069006C006900700020002D8F
:1013A80000200041005000490043000000000004F4
:1013B800030904C3000000000000000000AAAAAA54
:1013C800AAAAAAAAAAEEEEEEEEEEEEEEEEFEFFFF57
:1013D800FFFFFFFFFFFFFFFFFF7FBFDFEFF7FBFD13
:0B13E800FC7EBFDFEFF7FBFD7EB6CE02
:101EDF00FF18A4FF0DFBFF0009FF0FA9FF0009FF6B
:101EEF001F97FF002EFF0009FF2032FF1805FF1973
:101EFF003FFF1C30FF0009FF0009FF0009FF000929
:10176200AF34EF30E007C2AF121149D2AFAF33EF5F
:10177200131313541FFFEF30E027C2AFAF33EF5400
:10178200F7F533D2AF90700CE0FFEF4420FF90707A
:101792000CEFF090700CE0FFEF54DFFF90700CEF55
:1017A200F0AF33EFC4540FFFEF30E027C2AFAF33D7
:1017B200EF54EFF533D2AF90700CE0FFEF4440FFEF
:1017C20090700CEFF090700CE0FFEF54BFFF907040
:1017D2000CEFF0AF33EFC4135407FFEF30E023C236
:1017E200AFAF33EF54DFF533D2AFAF5FEF30E0127C
:1017F200D290AF5FEF54FEF55F120916753702758E
:0318020038002289
:10114900AF34EF54FEF534AF5DEF54BFF55D9070E9
:101159002C7420F0907020E0FF78A6A607907020EC
:10116900E0FF78A7A607907020E0FF7E0078A8A688
:101179000608A60778A8E6FE08E6FFEF7F00FE78D6
:10118900A8A60608A60778A8E6FE08E6FF9070203C
:10119900E0FD7C00EE4CFEEF4DFF78A8A60608A600
:1011A90007907020E0FF7E0078AAA60608A60778B7
:1011B900AAE6FE08E6FFEF7F00FE78AAA60608A6C3
:1011C9000778AAE6FE08E6FF907020E0FD7C00EEB5
:1011D9004CFEEF4DFF78AAA60608A607907020E0FE
:1011E900FF7E0078ACA60608A60778ACE6FE08E6FE
:1011F900FFEF7F00FE78ACA60608A60778ACE6FEEE
:1012090008E6FF907020E0FD7C00EE4CFEEF4DFFFC
:1012190078ACA60608A60778ACE6F55A08E6F55BA9
:1012290078AC7600087600AF5B7E0078ACA606083D
:10123900A60778ACE6FE08E6FFEF7F00FE78ACA6CD
:101249000608A607E55AF55B755A0078ACE6FE086C
:10125900E6FFEE455AFEEF455BFF78ACA60608A609
:101269000778A6E6FFEF5460F54178A7E6FFEF544B
:101279000FF542E541B440041213F322E541701E13
:10128900AF42EF75F003A424DFF582E4341EF58341
:0E129900E493FB740193FA740293F9121604A5
:0112A7002224
:1013F30078A7E6FFEF640C600302153778AAE6FED0
:1014030008E6FFEF8EF01215D71443710414187217
:1014130004000014BE78ACE6FE08E6FFEF64014E5C
:10142300701E90702C7401F090701C7401F0907019
:101433001DE4F09070207422F0121C931220FC2201
:10144300121D4590702CE4F0907020E0FF8F2790E0
:101453007020E0FF8F28907020E0FF8F299070208C
:10146300E0FF7E008E5A8F5B907020E0FFE4FCFD6E
:10147300FE8F3E8E3D8D3C8C3BAF3EAE3DAD3CACD6
:101483003B78081215878F3E8E3D8D3C8C3BAE5AC0
:10149300AF5BE4FCFDE53E4FF53EE53D4EF53DE536
:1014A3003C4DF53CE53B4CF53B907020E0FF8F2E27
:1014B3001220CCAF5FEF4420F55F2278A6E6FFEF62
:1014C300B4C0041220CC2278A6E6FFEF6440706417
:1014D30090702CE4F0907028E0FFEF4401FF9070CF
:1014E30028EFF0AF34EF20E044907018E0FCA3E065
:1014F300FDA3E0FEA3E0FFE5364FF536E5354EF5F7
:1015030035E5344DF534E5334CF533AF36AE35AD13
:1015130034AC3390701812159AAF33EF131313547E
:101523001FFFEF20E00EAF33EF30E0B722AF34EF11
:0515330054F7F534221D
:0100090022D4
:10002E0078A8E6FE08E6FFEF8EF01215D7005F0007
:10003E000100CC00020359000303CC000403D000DE
:10004E0005060B0006068E000709150008000008BD
:10005E00B0AF5FEF30E0087E127FA88E2F8F30AFEB
:10006E005FEF20E0087E127FBA8E2F8F30AE2FAF5B
:10007E00308F828E83E493FF7E008E178F189070E0
:10008E002C7401F090701C7412F090701DE4F0E569
:10009E001845176022AE2FAF308F828E83E493FF08
:1000AE00907020EFF0E5181518700215170530E561
:1000BE00307002052F80D8121C931220FC22AF3410
:1000CE00EF54FBF534755A00755B407E127FD68E69
:1000DE002F8F30AE2FAF308F828E83E493FF7E0052
:1000EE008E178F1890702C7401F078ACE6FE08E62F
:1000FE00FFC3E5189FE5179E405878ADE6FF907058
:10010E001CEFF078ACE6FE08E6FFEEFF7E00907086
:10011E001DEFF075170075180078ACE6FE08E6FFC7
:10012E00C3E5189FE5179E5022AE2FAF308F828EFB
:10013E0083E493FF907020EFF00530E530700205F8
:10014E002F0518E5187002051780CE121C93122089
:10015E00FC2278ACE6FE08E6FFC3EF9420EE940096
:10016E005003020344E51845176022AE2FAF308FBF
:10017E00828E83E493FF907020EFF0E518151870CF
:10018E000215170530E5307002052F80D8AF5FEFEE
:10019E0030E0087E127FE88E2F8F30AF5FEF20E0C9
:1001AE00087E127FF18E2F8F30AE2FAF308F828E62
:1001BE0083E493FF7E008E178F18E5184517602293
:1001CE00AE2FAF308F828E83E493FF907020EFF0CE
:1001DE00E5181518700215170530E5307002052F59
:1001EE0080D8AF5FEF30E0087E137F1D8E2F8F30EB
:1001FE00AF5FEF20E0087E137F2B8E2F8F30AE2F58
:10020E00AF308F828E83E493FF7E008E178F18E5BA
:10021E001845176022AE2FAF308F828E83E493FF86
:10022E00907020EFF0E5181518700215170530E5DF
:10023E00307002052F80D8AF5FEF30E0087E137F5D
:10024E00168E2F8F30AF5FEF20E0087E137F248E47
:10025E002F8F30AE2FAF308F828E83E493FF7E00D0
:10026E008E178F18E51845176022AE2FAF308F828C
:10027E008E83E493FF907020EFF0E518151870024E
:10028E0015170530E5307002052F80D8AF5FEF30BF
:10029E00E0087E137F018E2F8F30AF5FEF20E008D6
:1002AE007E137F0F8E2F8F30AE2FAF308F828E83C7
:1002BE00E493FF7E008E178F18E51845176022AE67
:1002CE002FAF308F828E83E493FF907020EFF0E596
:1002DE00181518700215170530E5307002052F80BD
:1002EE00D8AF5FEF30E0087E127FFA8E2F8F30AFDF
:1002FE005FEF20E0087E137F088E2F8F30AE2FAF7A
:10030E00308F828E83E493FF7E008E178F18E51850
:10031E0045176022AE2FAF308F828E83E493FF900D
:10032E007020EFF0E5181518700215170530E5303E
:10033E007002052F80D8907028E0FFEF4408FF90E0
:10034E007028EFF0121C931220FC227E137FB78EC2
:10035E002F8F30AE2FAF308F828E83E493FF7E00CF
:10036E008E178F1890702C7401F078ACE6FE08E6AC
:10037E00FFC3EF9518EE9517500978ACE6F5170800
:10038E00E6F518AF1890701CEFF090701DE4F0E5D4
:10039E001845176022AE2FAF308F828E83E493FF05
:1003AE00907020EFF00530E5307002052FE518153E
:1003BE00187002151780D8121C931220FC221200FE
:1003CE000922755A00755B0078A8E6FE08E6FF7EE6
:1003DE0000D3EF9401EE94004063907028E0FFEF9D
:1003EE004401FF907028EFF0AF34EF20E04790709B
:1003FE0018E0FCA3E0FDA3E0FEA3E0FFE5364FF519
:10040E0036E5354EF535E5344DF534E5334CF533FB
:10041E00AF36AE35AD34AC3390701812159AAF338B
:10042E00EF131313541FFFEF30E003020915AF3320
:10043E00EF30E0B422AF34EF54F7F534227E127F62
:10044E00FA8E2F8F30AE2FAF308F828E83E493FFD4
:10045E007E008E178F1890702C7401F078ACE6FE2B
:10046E0008E6FFC3E5189FE5179E405978ACE6F500
:10047E005A08E6F55BAF5B90701CEFF0E55AFF7E15
:10048E000090701DEFF075170075180078ACE6FE41
:10049E0008E6FFC3E5189FE5179E5022AE2FAF303A
:1004AE008F828E83E493FF907020EFF00530E5305D
:1004BE007002052F0518E5187002051780CE121C64
:1004CE00931220FC2278ACE6FE08E6FFC3EF9518E7
:1004DE00FFEE9517FE78ACA60608A607E518255B75
:1004EE00F55BE517355AF55AE51845176022AE2F1C
:1004FE00AF308F828E83E493FF907020EFF0E5187B
:10050E001518700215170530E5307002052F80D8CA
:10051E007E137F018E2F8F30AE2FAF308F828E8362
:10052E00E493FF7E008E178F1878ACE6FE08E6FF88
:10053E00C3E5189FE5179E406178ACE6FE08E6FF1E
:10054E00EF255BF55BEE355AF55AAF5B90701CEFFD
:10055E00F0E55AFF7E0090701DEFF07517007518CC
:10056E000078ACE6FE08E6FFC3E5189FE5179E503F
:10057E0022AE2FAF308F828E83E493FF907020EFE8
:10058E00F00530E5307002052F0518E518700205EC
:10059E001780CE121C931220FC2278ACE6FE08E6E1
:1005AE00FFC3EF9518FFEE9517FE78ACA60608A6CA
:1005BE0007E518255BF55BE517355AF55AAF5B90E5
:1005CE00701CEFF0E55AFF7E0090701DEFF0E518FD
:1005DE0045176022AE2FAF308F828E83E493FF904B
:1005EE007020EFF0E5181518700215170530E5307C
:1005FE007002052F80D8121C931220FC227E127FCF
:10060E00CC8E2F8F30AE2FAF308F828E83E493FF40
:10061E007E008E178F1890702C7401F078ACE6FE69
:10062E0008E6FFC3EF9518EE9517501978ADE6FF63
:10063E0090701CEFF090701DE4F078ACE6F51708A2
:10064E00E6F518800CAF1890701CEFF090701DE45A
:10065E00F0E51845176022AE2FAF308F828E83E4FF
:10066E0093FF907020EFF00530E5307002052FE516
:10067E001815187002151780D8121C931220FC2220
:10068E00755A00755B407E127FDF8E2F8F30AE2F36
:10069E00AF308F828E83E493FF7E008E178F18907B
:1006AE00702C7401F078ACE6FE08E6FFC3E5189FE7
:1006BE00E5179E405878ADE6FF90701CEFF078ACD1
:1006CE00E6FE08E6FFEEFF7E0090701DEFF0751758
:1006DE000075180078ACE6FE08E6FFC3E5189FE546
:1006EE00179E5022AE2FAF308F828E83E493FF90F1
:1006FE007020EFF00530E5307002052F0518E51873
:10070E007002051780CE121C931220FC2278ACE6E4
:10071E00FE08E6FFC3EF9420EE9400500302089B00
:10072E00E51845176022AE2FAF308F828E83E4938B
:10073E00FF907020EFF0E5181518700215170530B0
:10074E00E5307002052F80D87E127FE88E2F8F3015
:10075E00AE2FAF308F828E83E493FF7E008E178F85
:10076E0018E51845176022AE2FAF308F828E83E4C6
:10077E0093FF907020EFF0E518151870021517050D
:10078E0030E5307002052F80D87E137F1D8E2F8F9F
:10079E0030AE2FAF308F828E83E493FF7E008E17A4
:1007AE008F18E51845176022AE2FAF308F828E83DB
:1007BE00E493FF907020EFF0E518151870021517EE
:1007CE000530E5307002052F80D87E137F168E2FF0
:1007DE008F30AE2FAF308F828E83E493FF7E008EEC
:1007EE00178F18E51845176022AE2FAF308F828E07
:1007FE0083E493FF907020EFF0E518151870021542
:10080E00170530E5307002052F80D87E137F018EDC
:10081E002F8F30AE2FAF308F828E83E493FF7E000A
:10082E008E178F18E51845176022AE2FAF308F82C6
:10083E008E83E493FF907020EFF0E5181518700288
:10084E0015170530E5307002052F80D87E127FFA1D
:10085E008E2F8F30AE2FAF308F828E83E493FF7E3C
:10086E00008E178F18E51845176022AE2FAF308F08
:10087E00828E83E493FF907020EFF0E518151870C8
:10088E000215170530E5307002052F80D8907028BC
:10089E00E0FFEF4408FF907028EFF0121C93122037
:1008AE00FC2290702C7401F0907028E0FFEF440150
:1008BE00FF907028EFF0AF34EF20E044907018E016
:1008CE00FCA3E0FDA3E0FEA3E0FFE5364FF536E521
:1008DE00354EF535E5344DF534E5334CF533AF365D
:1008EE00AE35AD34AC3390701812159AAF33EF139A
:1008FE001313541FFFEF20E00EAF33EF30E0B7229B
:08090E00AF34EF54F7F5342279
:101F9700AF34EF54FBF53478A8E6FE08E6FFEEFF12
:101FA7007E00EF547FFF907000E0FEEE5480FEEE5F
:0B1FB7004FFF907000EFF01220CC22D2
:10180500AF34EF54FBF53478A8E6FE08E6FFEF4E5B
:101815007007751B001220CC2278A8E6FE08E6FFAB
:10182500EFB40015EEB4011178A8E6FE08E6FFEE68
:10183500FF7E008F1B1220CC2290702C7401F0903B
:101845007028E0FFEF4401FF907028EFF0AF34EF10
:1018550020E044907018E0FCA3E0FDA3E0FEA3E0C7
:10186500FFE5364FF536E5354EF535E5344DF534BE
:10187500E5334CF533AF36AE35AD34AC3390701837
:1018850012159AAF33EF131313541FFFEF20E00E19
:0F189500AF33EF30E0B722AF34EF54F7F5342222
:1020320090702C7401F0907020E51BF0907028E0F5
:10204200FFEF4408FF907028EFF0121C931220FC5F
:01205200226B
:100DFB0078A6E6FFEF540FF543E543640260030268
:100E0B000F2578A8E6FE08E6FFEF4E6003020F25DC
:100E1B0078AAE6FE08E6FFEF8EF01215D70E7400E7
:100E2B00000E8301000E9302000EA303000EB30409
:100E3B00000EC305000ED306000EE307000E6C80F8
:100E4B00000E7B81000E8B82000E9B83000EAB8409
:100E5B00000EBB85000ECB86000EDB870000000E5C
:100E6B00E990702C7401F0807590702CE4F0806E1A
:100E7B0090702C7403F0806690702C7402F0805E7E
:100E8B0090702C7405F0805690702C7404F0804E8A
:100E9B0090702C7407F0804690702C7406F0803E96
:100EAB0090702C7409F0803690702C7408F0802EA2
:100EBB0090702C740BF0802690702C740AF0801EAE
:100ECB0090702C740DF0801690702C740CF0800EBA
:100EDB0090702C740FF0800690702C740EF0907044
:100EEB0028E0FFEF54FEFF907028EFF0AF5EEF5459
:100EFB007FF55E907008E0FFEF54F7FF907008EFFE
:100F0B00F0907008E0FFEF4408FF907008EFF012CC
:100F1B0020CCAF23EF54FDF52322E543701A78A8BC
:100F2B00E6FE08E6FFEFB4000FEEB4010BAF23EFC4
:100F3B0054FEF5231220CC2290702C7401F090708B
:100F4B0028E0FFEF4401FF907028EFF0AF34EF2063
:100F5B00E044907018E0FCA3E0FDA3E0FEA3E0FFEB
:100F6B00E5364FF536E5354EF535E5344DF534E5DB
:100F7B00334CF533AF36AE35AD34AC33907018120D
:100F8B00159AAF33EF131313541FFFEF20E00EAF7F
:0D0F9B0033EF30E0B722AF34EF54F7F534F8
:010FA8002226
:1018A40078A6E6FFEFB4802290702C7401F090705B
:1018B4001C7402F090701DE4F09070207401F0909C
:1018C4007021E4F0121C931220FC78A6E6FFEFB41A
:1018D400812190702C7401F090701C7402F090704F
:1018E4001DE4F0907020E4F0907021E4F0121C9359
:1018F4001220FC78A6E6FFEF6482703E755A0075EC
:101904005B00AF23EFC313FFEF5401FF7E008E5A39
:101914008F5B90702C7401F090701C7402F09070C6
:101924001DE4F0AF5B907020EFF0E55AFF7E00906D
:0B1934007021EFF0121C931220FC2227
:100FA90078A6E6FFEF540FF543E5436402600302B8
:100FB90010C578A8E6FE08E6FFEF4E60030210C5EB
:100FC90078AAE6FE08E6FFEF8EF01215D710220088
:100FD900001031010010410200105103001061049A
:100FE90000107105001081060010910700101A8089
:100FF900001029810010398200104983001059849A
:10100900001069850010798600108987000000109A
:101019009790702C7401F0807590702CE4F0806EBC
:1010290090702C7403F0806690702C7402F0805ECE
:1010390090702C7405F0805690702C7404F0804EDA
:1010490090702C7407F0804690702C7406F0803EE6
:1010590090702C7409F0803690702C7408F0802EF2
:1010690090702C740BF0802690702C740AF0801EFE
:1010790090702C740DF0801690702C740CF0800E0A
:1010890090702C740FF0800690702C740EF0907094
:1010990028E0FFEF4401FF907028EFF0AF5EEF44C6
:1010A90080F55E907008E0FFEF54F7FF907008EF4D
:1010B900F01220CCAF23EF54FDF52322E543701A3B
:1010C90078A8E6FE08E6FFEFB4000FEEB4010BAF17
:1010D90023EF4401F5231220CC2290702C7401F0E7
:1010E900907028E0FFEF4401FF907028EFF0AF34D3
:1010F900EF20E044907018E0FCA3E0FDA3E0FEA31C
:10110900E0FFE5364FF536E5354EF535E5344DF575
:1011190034E5334CF533AF36AE35AD34AC3390707E
:101129001812159AAF33EF131313541FFFEF20E072
:0F1139000EAF33EF30E0B722AF34EF54F7F53499
:011148002284
:10193F0078A8E6FE08E6FFEF4E6060907028E0FFA3
:10194F00EF4401FF907028EFF0AF34EF20E04490A8
:10195F007018E0FCA3E0FDA3E0FEA3E0FFE5364F27
:10196F00F536E5354EF535E5344DF534E5334CF5C3
:10197F0033AF36AE35AD34AC3390701812159AAF15
:10198F0033EF131313541FFFEF20E039AF33EF3052
:10199F00E0B722AF34EF54F7F5342290702C740176
:1019AF00F090701C7401F090701DE4F0AF26EF20E2
:1019BF00E007907020E4F080069070207401F01220
:0619CF001C931220CC2243
:101C300078AAE6FE08E6FFEF4E701678A8E6FE08E2
:101C4000E6FFEFB4000BEEB40107AF26EF4401F559
:101C50002678AAE6FE08E6FFEFB40016EEB40112FD
:101C600078A8E6FE08E6FFEF4E7007AF26EF54FEB9
:101C7000F52678AAE6FE08E6FFEF4E701278A8E691
:101C8000FE08E6FFEF4E7007AF26EF54FEF5261272
:031C900020CC2243
:1020CC0090702C7401F0907028E0FFEF4402FF90A8
:0820DC007028EFF0121C9322A2
:101C9300AF34EF131313541FFFEF20E04490701879
:101CA300E0FCA3E0FDA3E0FEA3E0FFE5364FF5363D
:101CB300E5354EF535E5344DF534E5334CF533AFC5
:101CC30036AE35AD34AC3390701812159AAF33EF8E
:101CD300131313541FFFEF20E00EAF33EF30E0B0C8
:091CE30022AF34EF54F7F534226E
:1020FC0090702CE4F0907028E0FFEF4402FF907099
:07210C0028EFF0121D45222F
:101D4500AF34EF1313543FFFEF20E044907018E0D9
:101D5500FCA3E0FDA3E0FEA3E0FFE5364FF536E585
:101D6500354EF535E5344DF534E5334CF533AF36C1
:101D7500AE35AD34AC3390701812159AAF33EF13FE
:101D85001313541FFFEF20E00EAF33EF30E0B12205
:081D9500AF34EF54FBF53422DA
:101ADD00D310AF01C3C0D08F418C428D438B448A4C
:031AED00458946E2
:101AF00090702CE541F090701DE0FF7E008E428FCB
:101B000043E543754300F54290701CE0FF7E00EF13
:101B10002543F543EE3542F542854247854348E586
:101B2000481548AE4770021547FFEF4E601C907095
:101B300020E0FFAB44AA45A946EF121551740125D8
:0E1B400046F546E43545F54580D5AE42AF4347
:051B4E00D0D092AF228F
:0C1CEC008F418C428D438B448A45894611
:101CF80090702CE541F0AF4390701CEFF0E542FF87
:101D08007E0090701DEFF0854247854348E54815F1
:101D180048AE4770021547FFEF4E601CAB44AA451A
:101D2800A946121538FF907020EFF074012546F58A
:0C1D380046E43545F54580D5AE42AF438A
:011D4400227C
:10211300D29700D2960000000000C2970000000092
:0621230000C2960000223C
:10213C00C29700D2960000000000D2970000000069
:01214C002270
:021DEE008F5113
:101DF000755200E552C394085026AF52E551A8072A
:101E0000088002C333D8FCFFEF30E704D29780028A
:101E1000C29700D2960000000000C296055280D3FF
:101E20000000D2970000D296000000309704C20054
:081E30008002D200C2960000FE
:011E38002287
:101EAC00754900D297754A00E54AC39408501D0045
:101EBC00C2960000000000D2960000E54925E0F52E
:101ECC004930970205490000054A80DCC2960000A3
:021EDC00AF490C
:011EDE0022E1
:1020E400200104C2978002D297000000D29600001B
:0820F400000000C2960000226A
:102053008F628D63122113AF62121DEE200002C343
:1020630022AF63121DEE200002C32212213CD322B1
:0A1D9D008F4A8D4B8B4C8A4D894E06
:101DA700122113AF4A121DEE200002C322AF4B12BD
:101DB7001DEE200002C322755000E550C3954F5019
:101DC70021AB4CAA4DA94E121538FF121DEE20006B
:101DD70002C3227401254EF54EE4354DF54D0550ED
:061DE70080D812213CD35C
:011DED0022D3
:101F3D008F1C8B1D8A1E891F122113E51C04FF1295
:101F4D001DEE200002C322121EACAB1DAA1EA91F3E
:0E1F5D00EF121551D2011220E412213CD322C2
:0A1B53008F428D438B448A4589467A
:101B5D00122113AF42121DEE200002C322AF431219
:101B6D001DEE200002C322122113E54204FF121DB7
:101B7D00EE200002C322754800E54714FFE548C377
:101B8D009F5021121EACAB44AA45A946EF12155128
:101B9D00C2011220E474012546F546E43545F545AC
:101BAD00054880D5121EACAB44AA45A946EF1215C7
:0A1BBD0051D2011220E412213CD3A2
:011BC70022FB
:022092008F4A73
:10209400754C00E54CC3954A5012754B00E54BC393
:0C20A400943C5004054B80F5054C80E78F
:0120B000220D
:101FEA008F648D65E564D3941740037F00227B00DC
:101FFA007A007965754F01AD647F70121D9D7F0A65
:06200A001220927F01226A
:042010008F468D4723
:102014008546488547497B007A007948754F027D9B
:0D202400077F70121D9D7F0A1220927F0120
:01203100228C
:081E78008B418A4289438D442D
:101E8000754500E545C395445021E5452460FFAB09
:101E900041AA42A943121538FD12201074012543AE
:0B1EA000F543E43542F542054580D8CB
:011EAB002214
:1020B1007541007B007A0079417547017D017F7090
:0A20C100121B537F0A122092AF4158
:0120CB0022F2
:030000000219D50D
:0C19D500787FE4F6D8FD7581B3021A1C7F
:10153800BB010689828A83E0225002E722BBFE02B1
:09154800E32289828A83E49322E4
:10155100BB010689828A83F0225002F722BBFE0179
:02156100F32273
:10156300EB9FF5F0EA9E42F0E99D42F0E89C45F0DE
:011573002255
:10157400E8600FECC313FCED13FDEE13FEEF13FF55
:03158400D8F12279
:10158700E8600FEFC333FFEE33FEED33FDEC33FCC2
:03159700D8F12266
:0C159A00ECF0A3EDF0A3EEF0A3EFF022C4
:1015A600A8828583F0D083D0821215BD1215BD1294
:1015B60015BD1215BDE473E493A3C583C5F0C583B9
:1015C600C8C582C8F0A3C583C5F0C583C8C582C88F
:0115D60022F2
:1015D700D083D082F8E4937012740193700DA3A3A3
:1015E70093F8740193F5828883E473740293B5F0DA
:0D15F700067403936860E9A3A3A3A380D842
:061604008A838982E47371
:1019E10002160AE493A3F8E493A34003F68001F2FC
:1019F10008DFF48029E493A3F85407240CC8C33307
:101A0100C4540F4420C8834004F456800146F6DFD5
:101A1100E4800B0102040810204080902163E47EE1
:101A2100019360BCA3FF543F30E509541FFEE493CA
:101A3100A360010ECF54C025E060A840B8E493A391
:101A4100FAE493A3F8E493A3C8C582C8CAC583CABC
:101A5100F0A3C8C582C8CAC583CADFE9DEE780BE74
:01216A000074
:00000001FF
